:020000040000FA
:04000000CC303A289E
:08000800A000030EA100831209
:1000100005191128831601178312B2308100B0012F
:100020002C2883160113831203140B190310A80D37
:10003000A90DAA0DAB0DAC0DAC16FF302C02031DA3
:100040002C28FA302B02031D2C2831152A08AF006A
:100050002908AE002808AD008B100B11210E83007B
:06006000A00E200E0900B5
:0C007400203084008001840A80300402E7
:10008000031C3C28972183160C30850587018312B9
:10009000850187010730990000309A0010308316DF
:1000A0008E008312603083168F0083120030831617
:1000B00091009F008312C830831681008312313073
:1000C0009000003083168C00831210308B00362293
:1000D00081018E018F010B118B100B108C018B177E
:1000E0007F2031198B20B30B7D2803108519031451
:1000F000B90DF0303902031910218D2270286400E7
:100100003210B00A301F8A28AC01AB01AA01A90144
:10011000A801B001080031110130B7008B13203065
:10012000370783169B001C141A088312A400103092
:10013000370783169B001C141A088312A300A6001D
:100140000230A6060030370783169B001C141A08DD
:100150008312A200A7000130A7068B17321CB62815
:1001600022090339A200A309A409A50924082F0222
:10017000031D0A2923082E02031D0A2922082D0225
:10018000031D0A2901303702031DCB283D18CB2857
:100190003D143E14B22102303702031DD428BD188D
:1001A000D428BD143E14BE2103303702031DDD28C0
:1001B0003D19DD283D153E14CA2104303702031DC8
:1001C000E628BD19E628BD153E14D62105303702B4
:1001D000031DEF283D1AEF283D163E14E22106309C
:1001E0003702031DF828BD1AF828BD163E14ED216C
:1001F00007303702031D01293D1B01293D173E141D
:10020000F82108303702031D0A29BD1B0A29BD1732
:100210003E140322B70A09303702031808008E285B
:100220000130B600B300B400B500B7008501870106
:10023000B1137F20B30B4829031085190314B90D9E
:10024000F030390203196F29B40B48290130370205
:1002500003190E220230370203191322033037022A
:10026000031918220430370203191D220530370202
:1002700003192222063037020319272207303702DA
:1002800003192C2208303702031931229630B400AA
:10029000311D19293111321C52292D090339AD00A4
:1002A000AE09AF092F1C19298E018F010C1C1929C9
:1002B0000C102E1E19298B1320303707BB002F0876
:1002C000BA00822110303707BB002E08BA00822105
:1002D00000303707BB002D08BA0082218B1785013B
:1002E0008701B70AB60109303702031C19293622E3
:1002F00008003E1C08003E101030BB003D08BA004C
:10030000822108008B133A0883161C159A00831269
:100310003B0883169B0055309D00AA309D009C141D
:1003200064009C1890291C1183128B1708008316F7
:1003300010309B001C141A088312BD008316303045
:100340009B001C141A088312DE00FF30C800CA1577
:10035000CB15CC15CD15CE15CF15D015D115D21581
:10036000D3150800F130BD05FF30DE051130C4059E
:10037000C0000030C200C6005F100800F230BD05AA
:10038000FF30DE050230C405C0000030C200C600E8
:100390005F100800F430BD05FF30DE050630C405EF
:1003A000C0000030C200C6005F100800F830BD0574
:1003B000FF30DE051830C405C0000030C200C600A2
:1003C0005F1008001F30BD05C030DE058830C50550
:1003D000C1000030C300C70008002F30BD05C03089
:1003E000DE051030C505C1000030C300C70008009D
:1003F0004F30BD05C030DE053030C505C1000030CE
:10040000C300C70008008F30BD05C030DE05C03016
:10041000C505C1000030C300C700080010308506C4
:100420000230870608002030850600308706080065
:10043000213085060030870608000230850602302C
:1004400087060800003085060C308706080000305B
:1004500085060130870608000030850621308706B2
:100460000800003085061830870608003D18B221C4
:10047000BD18BE213D19CA21BD19D6213D1AE22160
:10048000BD1AED213D1BF821BD1B03220800B6015A
:10049000B301B4013C1C4F2ABC01BC14512ABC015D
:1004A0003C143C08B6006400552A562A572A582A9C
:1004B000592AFF30B41B8500B41F8501B30B532AA2
:1004C000B40B532A0310B60CB608031D532A003090
:1004D000BB003C08BA008221080005125C18051612
:1004E000DC1C8512DC1885165C1D05105C190514D2
:1004F000DC1D8510DC1985145C1E87105C1A8714BE
:10050000DC1E0711DC1A07155C1F07105C1B0714A3
:10051000DC1F8712DC1B871608008F0803190800F0
:100520008F0178308E00C80FB72CC80A441CBD2A32
:10053000461CAE2ACA1C9F2ACA014A15CB2A4A1D4C
:10054000A42ACA01CA15CB2ACA1DA92ACA014A1659
:10055000CB2A4A1ECB2ACA01CA14CB2A4A1DB32A67
:10056000CA014A16CB2ACA1DB82ACA014A16CB2A82
:100570004A1ECB2ACA01CA14CB2ACA1CC22ACA01E3
:100580004A15CB2A4A1DC72ACA01CA15CB2A4A1EB8
:10059000CB2ACA014A15C41CF22AC61CE32ACB1C6A
:1005A000D42ACB014B15002B4B1DD92ACB01CB15DF
:1005B000002BCB1DDE2ACB014B16002B4B1E002B34
:1005C000CB01CB14002B4B1DE82ACB014B16002B83
:1005D000CB1DED2ACB014B16002B4B1E002BCB0164
:1005E000CB14002BCB1CF72ACB014B15002B4B1D3A
:1005F000FC2ACB01CB15002B4B1E002BCB014B153E
:10060000441D272B461D182BCC1C092BCC014C1547
:10061000352B4C1D0E2BCC01CC15352BCC1D132BA3
:10062000CC014C16352B4C1E352BCC01CC14352B64
:100630004C1D1D2BCC014C16352BCC1D222BCC0177
:100640004C16352B4C1E352BCC01CC14352BCC1C29
:100650002C2BCC014C15352B4C1D312BCC01CC1542
:10066000352B4C1E352BCC014C15C41D5D2BC61DE6
:100670004E2BCD1C3F2BCD014D155F136B2B4D1D0C
:10068000442BCD01CD156B2BCD1D492BCD014D1626
:100690006B2B4D1E6B2BCD01CD146B2B4D1D532B96
:1006A000CD014D166B2BCD1D582BCD014D166B2B4F
:1006B0004D1E6B2BCD01CD146B2BCD1C622BCD01B0
:1006C0004D156B2B4D1D672BCD01CD156B2B4D1E85
:1006D0006B2BCD014D155F1B942B441E942B461E96
:1006E000852BCE1C762BCE014E15A22B4E1D7B2BBF
:1006F000CE01CE15A22BCE1D802BCE014E16A22BE5
:100700004E1EA22BCE01CE14A22B4E1D8A2BCE0143
:100710004E16A22BCE1D8F2BCE014E16A22B4E1E97
:10072000A22BCE01CE14A22BCE1C992BCE014E159E
:10073000A22B4E1D9E2BCE01CE15A22B4E1EA22B00
:10074000CE014E15C51DC92BC71DBA2BCF1CAB2B17
:10075000CF014F15D72B4F1DB02BCF01CF15D72B66
:10076000CF1DB52BCF014F16D72B4F1ED72BCF0147
:10077000CF14D72B4F1DBF2BCF014F16D72BCF1D1B
:10078000C42BCF014F16D72B4F1ED72BCF01CF1421
:10079000D72BCF1CCE2BCF014F15D72B4F1DD32BD3
:1007A000CF01CF15D72B4F1ED72BCF014F15451E8D
:1007B000FE2B471EEF2BD01CE02BD00150150C2C2C
:1007C000501DE52BD001D0150C2CD01DEA2BD001EB
:1007D00050160C2C501E0C2CD001D0140C2C501D7B
:1007E000F42BD00150160C2CD01DF92BD001501633
:1007F0000C2C501E0C2CD001D0140C2CD01C032C13
:10080000D00150150C2C501D082CD001D0150C2CEB
:10081000501E0C2CD0015015C51E332CC71E242C85
:10082000D11C152CD1015115412C511D1A2CD1016F
:10083000D115412CD11D1F2CD1015116412C511E17
:10084000412CD101D114412C511D292CD10151161B
:10085000412CD11D2E2CD1015116412C511E412C61
:10086000D101D114412CD11C382CD1015115412C6E
:10087000511D3D2CD101D115412C511E412CD101CE
:100880005115451F692C471F5A2CD21C4B2CD201E5
:100890005215DF13772C521D502CD201D215772C14
:1008A000D21D552CD2015216772C521E772CD20114
:1008B000D214772C521D5F2CD2015216772CD21DE8
:1008C000642CD2015216772C521E772CD201D214EE
:1008D000772CD21C6E2CD2015215772C521D732C02
:1008E000D201D215772C521E772CD2015215DF1B64
:1008F000A02CC51FA02CC71F912CD31C822CD30168
:100900005315AE2C531D872CD301D315AE2CD31DFC
:100910008C2CD3015316AE2C531EAE2CD301D31402
:10092000AE2C531D962CD3015316AE2CD31D9B2CED
:10093000D3015316AE2C531EAE2CD301D314AE2CC0
:10094000D31CA52CD3015315AE2C531DAA2CD301B7
:10095000D315AE2C531EAE2CD3015315792140086C
:10096000C4004108C5005F18DF145F1CDF10480891
:10097000C9000C304A05031D05120C304B05031D40
:1009800085120C304C05031D05100C304D05031D60
:1009900085100C304E05031D87100C304F05031DCC
:1009A00007110C305005031D07100C305105031DB5
:1009B00087120C305205031D07120C305305031D1E
:1009C000871149080E020318112D12304A05031D24
:1009D000051612304B05031D851612304C05031DFC
:1009E000051412304D05031D851412304E05031DEC
:1009F000871412304F05031D071512305005031DD3
:100A0000071412305105031D871612305205031DBD
:100A1000071612305305031D8715FF3048020319CE
:100A200008008F08031D08007F2049080E02031CE0
:100A3000112D18304A05031D051206304A05031D05
:100A4000051618304B05031D851206304B05031D96
:100A5000851618304C05031D051006304C05031D86
:100A6000051418304D05031D851006304D05031D76
:100A7000851418304E05031D871006304E05031DE2
:100A8000871418304F05031D071106304F05031D4D
:100A9000071518305005031D071006305005031DBB
:100AA000071418305105031D871206305105031D28
:100AB000871618305205031D071206305205031D14
:100AC000071618305305031D871106305305031D03
:040AD000871508007E
:084000000400030006000600A5
:02400E00CC33B1
:10420000010078007A007C007E007B0079007F004E
:104210007D007A0078007E007C007D007F007900C0
:104220000200F200F600FA00FE00F200F600FA00CA
:10423000FE00F200F600FA00FE00F200F600FA00BE
:10424000FF00050005000500050009000900090040
:1042500009000D000D000D000D00110011001100EE
:104260000100FF00FF00FF00FF00FF00FF00FF0054
:10427000FF00FF00FF00FF00FF00FF00FF00FF0046
:10428000FF007B00FF00FF00FF00FF00FF00FF00BA
:10429000FF00FF00FF00FF00FF00FF00FF00FF0026
:1042A000FF00FE00FF00FF00FF00FF00FF00FF0017
:1042B000FF00FF00FF00FF00FF00FF00FF00FF0006
:1042C000FF001100FF00FF00FF00FF00FF00FF00E4
:1042D000FF00FF00FF00FF00FF00FF00FF00FF00E6
:1042E000FF00FF00FF00FF00FF00FF00FF00FF00D6
:1042F000FF00FF00FF00FF00FF00FF00FF00DD00E8
:00000001FF
